:100000000C9417060C9447290C9474290C943F0601
:100010000C943F060C943F060C943F060C943F064C
:100020000C943F060C943F060C94C00C0C943F06B5
:100030000C943F060C943F060C943F060C943F062C
:100040000C94A1290C943F060C945B2D0C94962DD6
:100050000C943F060C943F060C943F060C943F060C
:100060000C943F060C943F069C1CA31CA31C9C1CD8
:10007000A31CA31CA31CA31CA31CA31CA31CA31C88
:10008000A31CA31CA31CA31CA31C111CA31CA31C0A
:10009000A31CA31CA31C741BA31CA31CA31CA31C98
:1000A000A31CA31CA31CA31CA31CA31CA31CA31C58
:1000B000A31CA31CA31C1D1C1D1C1D1C1D1C1D1CE6
:1000C0001D1C1D1C1D1C1D1CA31CA31CA31CA31C50
:1000D000A31CA31C791B1C1C1C1C1C1C1C1CA31C6F
:1000E0002D1C351C3D1C451C4D1C551C5D1C651CE8
:1000F0006F1C791C831C8D1CC01B801BA31CA31CA4
:10010000A31CA31C111CA31CA31CA31CA31CA31C89
:10011000A31CA31CA31C1B1C1B1C1B1C1B1CA31C07
:100120002D1C351C3D1C451C4D1C551C5D1C651CA7
:100130006F1C791C831C8D1CC01B801BA31CA31C63
:10014000A31CA31C111CD41CD41CD41CD41CD41C54
:10015000D41CD41CD41CD41CD41CD41CD41CD41C1F
:10016000F41DF41DF41DF41DF41DF41D1B1D251DAF
:100170002F1D391D9F1DA91DB71DC81D651ED51E2C
:10018000A61EAB1EB01EB51EBA1EBF1EC41ED51EB7
:10019000CF1EDA25EF25FB250426112637263F261C
:1001A00062264F26456E746572206D656E752E2E23
:1001B0002E00546F67676C6564206D6963726F50C1
:1001C000504D00546F67676C656420696E76657288
:1001D0007465642050504D2100546F67676C6564EE
:1001E000205458206D7574696E672100546F6767DD
:1001F0006C65642074656C656D657472792100505E
:10020000726F746F636F6C206572726F72207769A2
:1002100074682052580054696D656F757420776852
:10022000656E20636F6E6E656374696E6720746FB0
:1002300020525800507265737320616E79206B658F
:100240007920746F2063616E63656C00436F6E6E1E
:10025000656374696E6720746F2052582C20706F2C
:100260007765722075702074686520525820287751
:100270006974682062696E6420706C7567206966B5
:10028000206E6F74207573696E6720616C77617979
:10029000732062696E642900546F67676C6564201F
:1002A00027696D6D656469617465206F757470751B
:1002B000742700546F67676C65642027736C6176E0
:1002C00065206D6F64652700546F67676C656420F7
:1002D00027616C776179732062696E642700546FBF
:1002E00067676C65642050504D206368616E6E6571
:1002F0006C206C696D6974005365742052535349C6
:1003000020696E6A656374696F6E206368616E6EE2
:10031000656C2028303D3D64697361626C6529001D
:100320005365742050504D206D696E696D756D2058
:1003300073796E630053657420626561636F6E202C
:10034000696E74657276616C0053657420626561D4
:10035000636F6E2064656C6179005365742062651B
:1003600061636F6E206672657175656E6379206971
:100370006E20487A3A20303D64697361626C652C66
:100380002050783D504D52206368616E6E656C2040
:10039000782C2046783D465253206368616E6E6526
:1003A0006C2078005365742050574D2073746F7023
:1003B0002064656C61792028302064697361626C07
:1003C00065642C20312D323535203D3D20302E31D5
:1003D00073202D2035306D696E29005365742050CF
:1003E000504D2073746F702064656C6179202830E3
:1003F0002064697361626C65642C20312D3235355F
:10040000203D3D20302E3173202D2035306D696E1A
:100410002900536574206661696C736166652064A8
:10042000656C61792028302064697361626C656451
:100430002C20312D323535203D3D20302E3173209A
:100440002D2035306D696E29002A2A2A2A2A2A2A67
:100450002A2A2A2A2A2A2A2A2A2A2A2A2A2A2A2AFC
:100460002A2A2A2A2A2A0052582041636B656420CE
:100470002D2072657665727420737563636573737E
:1004800066756C21002A2A2A2A2A2A2A2A2A2A2A36
:100490002A2A2A2A2A2A2A2A2A2A2A2A2A2A2A2ABC
:1004A0002A2A002A2A2A2A2A2A2A2A2A2A2A2A2AD6
:1004B0002A2A2A2A2A2A2A2A2A2A2A2A2A2A2A2A9C
:1004C0000052582041636B6564202D207570646173
:1004D0007465207375636365737366756C21002A98
:1004E0002A2A2A2A2A2A2A2A2A2A2A2A2A2A2A2A6C
:1004F0002A2A2A2A2A2A2A2A2A2A2A2A0056616CE1
:1005000069642063686F69636573206172653A206E
:100510005B315D2D5B31365D20286368616E6E65F1
:100520006C20312D31362900536574206F7574703D
:10053000757420666F7220706F727420005B585D56
:100540002061626F7274206368616E6765732061F9
:100550006E64206578697420525820636F6E6669F6
:1005600067005B535D207361766520736574746901
:100570006E677320746F205258005B525D20726565
:10058000766572742052582073657474696E67734F
:1005900020746F2064656661756C747300557365B3
:1005A000206E756D62657273205B312D445D207421
:1005B0006F206564697420706F727473205B452DC1
:1005C000515D20666F722073657474696E67730085
:1005D000202D20726563656976657220636F6E6693
:1005E0006967757261746F722C207278207377203E
:1005F000000A0A6F70656E4C52536E672000536597
:10060000742073657269616C2062617564726174D3
:10061000653A200056616C69642063686F696365A0
:10062000733A2031202D20342B34202F2032202DDE
:100630002038202F2033202D20382B34202F203419
:10064000202D203132202F2035202D2031322B3407
:10065000202F2036202D203136005365742043682A
:10066000616E6E656C20636F6E6669673A20005339
:1006700065742044617461726174652028302D3284
:10068000293A200053657420486F70206368616EBA
:100690006E656C7320286D61782032342C20736570
:1006A0007061726174656420627920636F6D6D6141
:1006B00073292076616C69642076616C756573209E
:1006C000312D3235353A2000536574206368616EF0
:1006D0006E656C2073706163696E672028783130B5
:1006E0006B487A293A200053657420524620706F77
:1006F0007765722028302D37293A20005365742001
:100700005246206D616769632028686578292065F5
:100710002E672E20307844454144463030443A20FC
:10072000005365742062617365206672657175653A
:100730006E63792028696E20487A293A20005B5A36
:100740005D20656E74657220726563656976657299
:1007500020636F6E66696775726174696F6E20756C
:1007600074696C79005B465D20646973706C6179B3
:100770002061637475616C206672657175656E6366
:100780006965732075736564005B525D2063616CFD
:1007900063756C6174652072616E646F6D206B654A
:1007A0007920616E6420686F70206C697374005BDF
:1007B000495D207265696E697469616C697A65204A
:1007C00073657474696E677320746F20736B6574DE
:1007D00063682064656661756C7473005B585D20A6
:1007E000726576657274206368616E6765732061F7
:1007F0006E642065786974206D656E75005B535D6D
:1008000020736176652073657474696E67732074F4
:100810006F20454550524F4D20616E6420657869C8
:1008200074206D656E7500557365206E756D62651B
:100830007273205B302D395D20746F20656469749C
:1008400020706172616D657465727300202D205394
:10085000797374656D20636F6E6669677572617414
:10086000696F6E000A0A6F70656E4C52536E672096
:10087000005129204F7574707574206265666F721F
:1008800065206C696E6B20283D465329203A200074
:10089000502920536C617665206D6F646520286552
:1008A00078706572696D656E74616C293A20004FCD
:1008B000292054696D65642042494E4420617420AA
:1008C0007374617274757020203A20004E29205094
:1008D000504D206F7574707574206C696D69746506
:1008E0006420202020203A200044495341424C45B6
:1008F00044004D292050504D205253534920746FCD
:10090000206368616E6E656C202020203A20004CC8
:10091000292050504D206D696E696D756D20737979
:100920006E63202875732920203A200044495341E2
:10093000424C4544004B29204661696C73616665F1
:1009400020626561636F6E20696E74762E20283197
:100950002D32353573293A20004A29204661696CC9
:100960007361666520626561636F6E2064656C61AA
:10097000792028302D323535203D3E20313073200E
:100980002D203135306D696E293A200049292046E5
:1009900061696C7361666520626561636F6E206674
:1009A00072712E203A200048292050574D20737430
:1009B0006F702064656C6179202020202020203A0F
:1009C000200047292050504D2073746F70206465BB
:1009D0006C6179202020202020203A200046292008
:1009E0004661696C736166652064656C617920207D
:1009F00020202020203A200050574D206368616E4F
:100A00006E656C200066756E6374696F6E3A2000C7
:100A10002920706F72742000506F776572546F7761
:100A2000657200445446205548462033322D626991
:100A3000742031306368004F70656E4C52536E679E
:100A40005258206D696E6920342F36636800466CF9
:100A50007974726F6E2F4F72616E676552582055B0
:100A600048462038636800525820747970653A20EF
:100A70000044697361626C656400487A00203D3D02
:100A8000200043616C63756C617465642070616300
:100A90006B657420696E74657276616C3A200042F1
:100AA00029204D6963726F202868616C6629205087
:100AB000504D202020203A00412920496E76657251
:100AC0007465642050504D20696E20202020203A0B
:100AD000003029204D7574652062757A7A65722020
:100AE000286D6F73746C79293A0039292053657227
:100AF00069616C2062617564726174653A00736D3E
:100B0000617274506F7274004672536B7900547244
:100B1000616E73706172656E740044697361626CBA
:100B200065640038292054656C656D657472793A86
:100B300020202020202020003729204368616E6E6D
:100B4000656C20636F6E6669673A20200036292045
:100B500044617461726174652028302D32293A2015
:100B6000202000352920486F70206368616E6E6513
:100B70006C733A2020202020003429204368616EC5
:100B80006E656C2073706163696E673A2020003374
:100B90002920524620706F7765722028302D372922
:100BA0003A202020003229205246206D6167696377
:100BB0003A202020202020202020003129204261BE
:100BC0007365206672657175656E63793A202020C1
:100BD0000000000000240027002A0000000000257B
:100BE0000028002B0000000000230026002900043C
:100BF00004040404040404020202020202030303C4
:100C000003030301020408102040800102040810BD
:100C1000200102040810200000000700020100006B
:100C20000304060000000000000000003E2F112415
:100C30001FBECFEFD8E0DEBFCDBF13E0A0E0B1E034
:100C4000EEEBF0E602C005900D92A839B107D9F796
:100C500016E0A8E9B3E001C01D92AB35B107E1F79A
:100C60001CE0CEE2DCE004C02297FE010E943A3094
:100C7000CC32D107C9F70E94832F0C945D300C94BD
:100C80000000A0E0B0E0E7E4F6E00C940930EC01ED
:100C9000A880B980CA80DB80A114B104C104D1044A
:100CA00041F484E2A82E89EDB82E8BE5C82E87E0AA
:100CB000D82EC601B5012DE133EF41E050E00E948E
:100CC000E62F27EA31E440E050E00E94922F7B01BA
:100CD0008C01C601B5012DE133EF41E050E00E94E7
:100CE000E62FCA01B9012CEE34EF4FEF5FEF0E94FF
:100CF000922F6E0D7F1D801F911F97FF04C06150C2
:100D0000704080409048688379838A839B839B01ED
:100D1000AC015F77B901CA01CDB7DEB7EAE00C9448
:100D200025300E944106089581EB92E00E94410621
:100D300008956093B1027093B2028093B3029093CE
:100D4000B4020895A0E0B0E0E8EAF6E00C940230C6
:100D5000EC012B016A016115710519F0FB0191830A
:100D60008083C114D10449F0C6010297839728F00B
:100D700020E030E040E050E0DCC0A9908A2D90E017
:100D80000E945230892BC9F7FDE2AF1621F4A990D9
:100D90003324339405C08BE2A81609F4A9903324B8
:100DA000C114D10421F0E0E1CE16D10411F5F0E335
:100DB000AF1669F48881883711F0883541F4A9802D
:100DC000229682E0382A20E1C22ED12C12C0C11412
:100DD000D10479F4E0E3AE1659F199E9E92E99E9E5
:100DE000F92E99E9092F99E1192F8AE0C82ED12C03
:100DF0003AC0FAE0CF16D10491F080E1C816D104D0
:100E000029F0E8E0CE16D104F9F415C0BFEFEB2EBF
:100E1000BFEFFB2EBFEF0B2FBFE01B2F24C0A9E9B4
:100E2000EA2EA9E9FA2EA9E90A2FA9E11A2F1BC077
:100E3000F8E0CF2ED12CEFEFEE2EEFEFFE2EEFEFFE
:100E40000E2FEFE11E2F0FC09601442737FD40956E
:100E5000542F6FEF7FEF8FEF9FEF0E94C42FC901D8
:100E6000DA017C018D0120E030E040E050E060E0FC
:100E70003601882477FC8094982C70EDB72EBA0C3C
:100E8000F9E0FB1570F48A2D81548A3118F499EC3D
:100E9000B92E06C08A2D81568A3148F589EAB82EC6
:100EA000BA0C8B2D90E08C159D050CF56F3FE9F089
:100EB000E216F30604071507B8F0CA01B901A40148
:100EC00093010E94922F9B01AC018B2D90E0A0E03A
:100ED000B0E0280F391F4A1F5B1F281739074A0740
:100EE0005B0710F061E001C06FEFA990C6CF41141D
:100EF000510451F0662311F0219703C031FE04C064
:100F00002297F201D183C08330FE07C050954095EF
:100F1000309521953F4F4F4F5F4F67FF0AC082E2E8
:100F200090E090935A06809359062FEF3FEF4FEFD2
:100F30005FEFB901CA01CDB7DEB7E1E10C941E3015
:100F4000FC0188279927E89421912032E9F3293080
:100F500010F02E30C8F32B3241F02D3239F4689462
:100F600004C00E94F507820F911D219120532A3061
:100F7000C0F31EF4909581959F4F089548E953E082
:100F80000E94C3070895009731F4DA018D919C9176
:100F9000009709F40EC0DC01FB013D912191222351
:100FA00019F03217C9F3FACF332331F4DA011D9265
:100FB0001C928827992708951197AF93BF93FB013F
:100FC0003D912191321771F4332321F48827992719
:100FD000119702C01E921196FA01A193B0839F91BE
:100FE0008F910895222369F7EACF7AE0979F902D99
:100FF000879F802D910D1124089580919A0381304F
:1010000019F482E080939A0380919A03833019F453
:1010100084E080939A030895E3E0F0E089E0809310
:101020005700849190E08670863009F491E0892F12
:1010300008951F93182F0E940C08882379F09FB7FA
:1010400081E08093A105F894A89588E180936000E1
:1010500010936000112309F0A8959FBF1F91089578
:10106000382F20E080913305909134058227932713
:1010700040E061E270E19C01220F331F97FF04C042
:10108000C9018627972701C0C9014F5F483099F7EA
:101090009093340580933305089587E38093D003BC
:1010A00080E092ECA1E0B0E08093D1039093D20372
:1010B000A093D303B093D40387E08093DD0380EC47
:1010C0009AECA9E8B6E38093D5039093D603A09356
:1010D000D703B093D80385E08093DE038DEE9EEFB7
:1010E000ADEABEED8093D9039093DA03A093DB03BE
:1010F000B093DC03AFEDB3E080E090E0863010F019
:10110000E0E004C0FC01EF57FC4FE081ED93019655
:101110008831910599F782E08093F7038AE0809304
:10112000F803089580EC97EFAAEBB7E380939D0353
:1011300090939E03A0939F03B093A00380E090E060
:10114000A0E0B0E58093A1039093A203A093A30332
:10115000B093A403E5EAF3E080E081938F5F8031F0
:10116000E1F708958436910520F4BC0180E090E019
:1011700025C08E3B910550F48A559040BC0180E01B
:1011800090E02AE030E040E050E016C0823D91055A
:1011900050F4845B9040BC0180E090E024E630E0B5
:1011A00040E050E009C08D5C9040BC0180E090E0E0
:1011B00028E532E040E050E00E94922F24E630E043
:1011C00040E050E00E94922F089590E08C599F4F8C
:1011D0000E94B2080895DC019896EC91F0E0E77067
:1011E000F070E758FC4F808108958F929F92AF92E4
:1011F000BF92CF92DF92EF92FF920F931F938C01D9
:101200000E94EB08D80197962C9130E043E150E022
:10121000249FF001259FF00D349FF00D1124EB5415
:10122000FD4F80809180A280B38090E00F96AA2726
:1012300097FDA095BA2FBC01CD0120E43FE14DE719
:1012400050E00E94922FA50194010E94C42F6901D1
:101250007A0180ED97E0A0E0B0E0C80ED91EEA1E4A
:10126000FB1ED80198968C91887181F060E07EEE2B
:101270008AEB9BE0A50194010E94C42F28513C4FAA
:101280004F4F5F4FC20ED31EE41EF51E87EE93E054
:10129000A0E0B0E0C80ED91EEA1EFB1EC701B601D1
:1012A00028EE33E040E050E00E94C42FCA01B901AB
:1012B00028EE33E040E050E00E94922F1F910F9102
:1012C000FF90EF90DF90CF90BF90AF909F908F9066
:1012D00008958F3F910509F010F480E0089522E011
:1012E0008030920710F481E008958050934010F010
:1012F00083E0089582E00895CF92DF92FF920F93EA
:101300001F93CF93DF93F82FEB016A01182F1695E7
:10131000E0E088819981D6018C938A819B81119626
:101320008C9311978C819D8112968C9312978E814C
:101330009F8113968C931397288139814A815B8111
:101340006C817D818E819F819295990F990F907C00
:10135000832F8370982B852F8370880F880F982B8D
:10136000872F83708295807F982B14969C9385E0BD
:1013700090E0C80ED91E2896EF5F1E1750F6F0FFBA
:1013800021C0888199810E946909F82E8A819B81F8
:101390000E946909182F8C819D810E946909082F7C
:1013A0008E819F810E946909F294FF0CFF0C70EC02
:1013B000F7221295107F1F29182B000F000F012B09
:1013C000D6010C93DF91CF911F910F91FF90DF9089
:1013D000CF90089523E08032920718F420E030E0A7
:1013E00026C023E0883E920748F49C012F513340E9
:1013F00054E0369527955A95E1F719C027E0803DCE
:10140000920720F49C012C5D334011C028E08839FC
:10141000920718F02FEF33E00AC09C01285C374098
:1014200044E0369527954A95E1F72D503C4FC90188
:1014300008958C30910548F49C0174E0220F331F0D
:101440007A95E1F7285D3C4F17C023E0843F92076F
:1014500020F49C0124523C4F0FC024E080309207BE
:1014600018F020E938E008C09C012657334F64E0AB
:10147000220F331F6A95E1F7C90108959C01369543
:10148000279525753575821B930B9C0136952795FD
:10149000369527952373337383739373280F391FFE
:1014A000C901E4E096958795EA95E1F7820F931FCD
:1014B0008F709F7021E031E0AC01429FC001439FDB
:1014C000900D529F900D1124892F0895882339F093
:1014D0002D9800002B9A00002D9A000008952D9859
:1014E00000002B9800002D9A000008952D9A00000E
:1014F00083B12D98000090E0B4E096958795BA9559
:10150000E1F7817008950F931F93082F5C9A2D982F
:101510005C9810E0802F80780E94660A000F1F5FA1
:101520001830C1F72D981F910F9108958F770E9461
:10153000830A08950F931F93082F10E0802F80785F
:101540000E94660A000F1F5F1830C1F72D981F9187
:101550000F9108950F931F932D9880E000E0182FAE
:10156000110F0E94760A810F0F5F0830C1F71F919B
:101570000F9108950E94960A0E94AA0A5C9A089503
:101580001F93162F80680E94830A812F0E949A0A57
:101590005C9A1F9108951F931091D9031827E0EDCD
:1015A000F3E0E80FF11D89E767850E94C00A8DE32B
:1015B000612F0E94C00A82E4612F0E94C00A1F911D
:1015C000089586E20E94BA0A08950F931F938C0132
:1015D0008CE1F80164810E94C00A8DE1F801658107
:1015E0000E94C00A8EE1F80166810E94C00A80E272
:1015F000F80167810E94C00A81E2F80160850E94BB
:10160000C00A82E2F80161850E94C00A83E2F80103
:1016100062850E94C00A84E2F80163850E94C00AC4
:1016200085E2F80164850E94C00A8AE2F8016585B6
:101630000E94C00A8EE6F80166850E94C00A8FE605
:10164000F80167850E94C00A80E7F80160890E945E
:10165000C00A81E7F80161890E94C00A82E7F801A7
:1016600062890E94C00A1F910F910895EF92FF9224
:101670000F931F93CF93DF937B018C01603028E39E
:1016800072072CE982072CE1920728F520E836E959
:1016900048E950E00E94C42FE9016897B90180E051
:1016A00090E020E839E647E65FEF0E94922F6E0D4A
:1016B0007F1D801F911F32E0660F771F881F991FC3
:1016C0003A95D1F721E732E040E050E00E94C42F84
:1016D000890180E421C020E03DE241E351E00E9425
:1016E000C42FE9016897B90180E090E020E033ED74
:1016F0004EEC5EEF0E94922F6E0D7F1D801F911F9A
:10170000660F771F881F991F21E732E040E050E005
:101710000E94C42F890180E69E012F71622F680FFD
:1017200085E70E94C00A86E7612F0E94C00A87E70A
:10173000602F0E94C00ACDB7DEB7E6E00C942930D6
:101740009F92AF92BF92CF92DF920F93DF93CF938E
:1017500000D000D0CDB7DEB7982E83E00E94BA0A41
:101760008093F90384E00E94BA0A8093FA0386E02A
:1017700060E00E94C00A87E061E00E94C00A89E040
:101780006FE70E94C00A8AE065E00E94C00A8BE011
:1017900062E10E94C00A8CE065E10E94C00A8DE00F
:1017A0006DEF0E94C00A8EE060E00E94C00A99209E
:1017B00019F084E193E008C08091F70323E1829F50
:1017C000C00111248B549D4F0E94E50A80E36CE810
:1017D0000E94C00A82E36FE00E94C00A83E362E4D1
:1017E0000E94C00A84E36AE00E94C00A85E36AE2BC
:1017F0000E94C00A86E36DE20E94C00A87E364ED9E
:101800000E94C00A88E360E00E94C00A89E360E0A9
:101810000E94C00A992049F065E8A62E61ECB62E18
:1018200061ECC62E6EEDD62E08C0A090D903B09004
:10183000DA03C090DB03D090DC030AE38D2D9927F7
:10184000AA27BB2789839A83AB83BC83802F6981B6
:101850000E94C00A802F8B5F69810E94C00ADC2C25
:10186000CB2CBA2CAA240F5F0E3341F783E46FEF21
:101870000E94C00A84E46FEF0E94C00A85E46FEF03
:101880000E94C00A86E46FEF0E94C00A992019F0F6
:101890008DE666E003C08DE66091DD030E94C00A1C
:1018A00089E760E00E94C00A8AE76091DE030E9437
:1018B000C00A83E760E00E94C00A84E760E00E94FB
:1018C000C00A992029F060EC7AEC89E896E308C018
:1018D0006091D5037091D6038091D7039091D8037E
:1018E0000E94360B0F900F900F900F90CF91DF91C9
:1018F0000F91DF90CF90BF90AF909F90089587E0B9
:1019000061E00E94C00A8EE764E20E94C00A88E09B
:1019100063E00E94C00A88E060E00E94C00A87E09D
:1019200065E00E94C00A85E062E00E94C00A83E090
:101930000E94BA0A8093F90384E00E94BA0A809355
:10194000FA030895582F40919E04842F90E0FC01E3
:10195000EF70F0709F012F5F3F4F74E09595879572
:101960007A95E1F72817390751F0E257FB4F50837A
:10197000842F8F5F8F70407F842B80939E04089507
:101980001F920F920FB60F9211241F932F933F9324
:101990004F935F936F937F938F939F93AF93BF9377
:1019A000CF93DF93EF93FF93C0918600D091870090
:1019B0002091E0043091E1048091BF04882309F074
:1019C00062C0BE01621B730B2091A1033091A20380
:1019D0004091A3035091A40325FD02C0769567951D
:1019E00089E0653C7807B8F1809147031CE1569582
:1019F0004795379527951A95D1F72115310541055A
:101A0000510521F421E030E040E050E090E0A0E01A
:101A1000B0E0281739074A075B07D0F480914703E5
:101A20008F3FB1F020E00EC0E22FF0E0EE0FFF1F7D
:101A3000DF01A054BB4F8D919C91E95DFC4F9183D8
:101A400080832F5F80914703281770F31092BE04A4
:101A50001092470318C082E06D3B780760F18091D7
:101A60004703803140F510914703CB010E94EA09FA
:101A7000E12FF0E0EE0FFF1FE054FB4F91838083D6
:101A80001F5F10934703D093E104C093E004FF91DC
:101A9000EF91DF91CF91BF91AF919F918F917F9106
:101AA0006F915F914F913F912F911F910F900FBEBA
:101AB0000F901F9018958FEF80934703E4CF83E03A
:101AC000809380008AE9809381008091A10386FD44
:101AD00005C0809181008064809381008FEF9FEF2B
:101AE000909389008093880080916F00806280933A
:101AF0006F0008956F3018F086958058089589E03A
:101B0000689F802D11240895882319F460E071E006
:101B100002C063E071E087E396E00E94462D0895DD
:101B2000A0E0B0E0E6E9FDE00C940B30182F0E9435
:101B3000F7299B01AC0180912D0590912E05A09174
:101B40002F05B091300569017A01C81AD90AEA0A4D
:101B5000FB0AD701C60189589341A040B04010F05C
:101B600010922C0520932D0530932E0540932F05C0
:101B7000509330052091BF04822F81508230E8F5C8
:101B800080912C05882309F44FC1813011F482E043
:101B9000BCC1803108F035C1E82FF0E0E054FB4FC4
:101BA00010838F5F80932C05803109F0B0C1A2ECC7
:101BB000B4E0213039F41196EC911197E695E69551
:101BC0008C9109C08D919C911197E92FE695E6952E
:101BD000E69596958795E03140F4F0E090E0EE0FC1
:101BE000FF1FE95DFC4F918380831092BE04129623
:101BF00084E0A03DB807E9F68AC1233009F004C1AA
:101C000080912C05882321F41F3009F080C10CC17C
:101C1000883130F4E82FF0E0E154FB4F108374C1B9
:101C2000883109F0EEC0112309F0EBC0C0E0D0E02C
:101C30000BE010E0DE0163E0AA0FBB1F6A95E1F73D
:101C4000C09FB001C19F700DD09F700D1124FB018A
:101C5000E054FB4F80812181922F97709595879555
:101C6000FD01EE0FFF1FE95DFC4F91838083FB01B7
:101C7000EF53FB4F30813695369536952181422FB3
:101C80004295440F407E842F832B269526952695DA
:101C9000922F977095958795FD01EE0FFF1FE75DD9
:101CA000FC4F91838083FB01EE53FB4F8081829533
:101CB0008695869583704181942F990F990F292FCE
:101CC000282B429546954695437082818170880FF6
:101CD000880F382F342B35952795FD01EE0FFF1F08
:101CE000E55DFC4F31832083FB01EC53FB4F3081DA
:101CF00036952181422F479544274795842F832B82
:101D00002695922F977095958795FD01EE0FFF1FF1
:101D1000E35DFC4F91838083FB01EB53FB4F3081EC
:101D200032953F702181422F4295407F842F832B33
:101D300022952F70922F977095958795FD01EE0F44
:101D4000FF1FE15DFC4F91838083FB01EA53FB4F52
:101D50008081881F8827881F4181942F990F292F00
:101D6000282B441F4427441F82818370880F382FFB
:101D7000342B35952795FD01EE0FFF1FEF5CFC4FCF
:101D800031832083FB01E853FB4F30813695369534
:101D90002181422F4295440F440F407C842F832B96
:101DA00026952695922F977095958795AA0FBB1F1C
:101DB000FD01ED5CFC4F9183808367537B4FFB01FA
:101DC00020812295269527704181342F330F330FC0
:101DD000330F832F822B942F92959695977095951C
:101DE0008795AB5CBC4F11969C938E932196C23025
:101DF000D10509F01FCF8091D60483FD02C0109257
:101E0000BE0410922C0583C0243009F080C040919C
:101E10002C05442359F4183AB1F410923405109269
:101E2000330588EA0E94300881E06FC0413019F420
:101E30001093310504C0423031F410933205812FE4
:101E40000E9430085DC060913205262F30E0220FDD
:101E5000331FE42FF0E0C90102968E179F0734F07C
:101E6000433268F7E354FB4F1083E9CF2D5F3F4FB8
:101E70004091330550913405E217F30749F4912F4F
:101E800080E048275927509334054093330538C0E4
:101E9000812F90E04817590789F5809131058130ED
:101EA00069F5613118F080E180933205D0903205F8
:101EB00040ECE42E44E0F42E00E010E01BC0F701FB
:101EC000D081C0E0818190E08C2B9D2B33E09695F2
:101ED00087953A95E1F70E94EA09F801EE0FFF1F96
:101EE000E95DFC4F918380830F5F1F4F82E090E09C
:101EF000E80EF91E0D1518F31092BE0410922C0571
:101F000080912C05882319F08F5F80932C05CDB725
:101F1000DEB7E8E00C942730FF920F931F93CF9326
:101F2000DF93182F092FF62E8EE30E94C00A212F6F
:101F3000302FC901EC0110E005C08FE769910E94C4
:101F4000C00A1F5F1F15C8F385E064E00E94C00A45
:101F500083E00E94BA0A8093F90384E00E94BA0ADF
:101F60008093FA030E94F7296093FB037093FC03AC
:101F70008093FD039093FE0387E069E00E94C00A0E
:101F800081E080939A03CDB7DEB7E5E00C942A3068
:101F90000E948C0F80919A038130D9F40E94F72916
:101FA0002091FB033091FC034091FD035091FE030F
:101FB000621B730B840B950B605A764881409040EE
:101FC00040F4E8CF87E396E067E071E00E94462D99
:101FD000089580919A038130A9F3089587E396E0EC
:101FE0006EE70E94FE2E0895A0E0B0E0EAEFFFE069
:101FF0000C940A306C0187E396E06EE70E94FE2E97
:10200000760100E010E0C0E0D0E0B0E2BB2E0AC0F4
:102010000830110521F49E012095F60120870894CF
:10202000E11CF11CF7016081862F8D57823040F44E
:1020300087E396E06DE70E94FE2EF70160816B2535
:1020400087E396E00E94FE2E0115110551F0F7017D
:1020500080819E01280F311DC32FDD27C20FD31FA2
:10206000D0700F5F1F4F0930110591F6CDB7DEB765
:10207000E9E00C942630A9E0B0E0E1E4F0E10C9452
:102080001130382FE62F8091A30490E0019664E28E
:1020900070E00E94B12F982F8093A30488E9898370
:1020A00080E18A83913071F0913028F0923099F07C
:1020B0009330E1F416C085E08B8381EF8C832F5F32
:1020C0002D8317C09B8381EF8C8384E6489FC001DA
:1020D00011249D830EC084E08B8381EF8C833D832C
:1020E00008C09B8381EF8C83ED8303C00E94EE0FB9
:1020F00004C0CE0101960E94F40F2996E2E00C94F0
:102100002D300F931F93CF93DF93182F092F87E361
:1021100096E06EE70E94FE2E212F302FC901EC01C0
:1021200010E000E288818D57823040F487E396E02A
:102130006DE70E94FE2E88818027888387E396E0E2
:1021400069910E94FE2E1F5F193061F787E396E0C8
:102150006EE70E94FE2EDF91CF911F910F9108959F
:10216000A9E0B0E0E6EBF0E10C941130382F80915B
:10217000A304882379F48EEF89833A836B83842FB9
:1021800090E0959587958C832D83198618861F82FC
:102190001E822FC040919E04842F90E09C012F70DE
:1021A000307054E0959587955A95E1F7821793071B
:1021B00021F18DEF89831A821B82DE01149620E0C3
:1021C00008C0E257FB4F80818D93405F2F5F263020
:1021D00069F0842F90E0FC0134E0F595E7953A959D
:1021E000E1F78F709070E817F90759F740939E0454
:1021F0002A83CE0101960E9481108091A30490E071
:10220000019666E070E00E94B12F8093A3042996A6
:10221000E2E00C942D309F92AF92BF92CF92DF926A
:10222000EF92FF920F931F93B82EA62ED42EC22E9C
:10223000902E0E94F7297B018C0180918D042091C2
:102240009F043091A0044091A1045091A2048823DE
:10225000B1F0D801C701821B930BA40BB50B815EB3
:102260009E42A040B04020F12C2DDC1408F42D2D0E
:102270008B2D6A2D422F292D0E943B1011C0D801B1
:10228000C701821B930BA40BB50B81539547A0404C
:10229000B04070F08B2D6A2D4D2D2C2D0E94B0106A
:1022A000E0929F04F092A0040093A1041093A20472
:1022B0001F910F91FF90EF90DF90CF90BF90AF9064
:1022C0009F90089587E396E0609100040E94FE2E9F
:1022D00008951F93182F87E396E0612F0E94FE2E2A
:1022E000809100048127809300041F9108951F931B
:1022F000192F0E946911812F0E9469111F91089561
:10230000DF92EF92FF920F931F93D82E7B011092D2
:10231000000407E316E0C80165EB0E94FE2EC80129
:1023200062E60E94FE2E8D2D0E946911C7010E9457
:1023300077111F910F91FF90EF90DF900895E82F94
:10234000F0E0E456FC4FE185E03158F4F894F0E019
:10235000EE0FFF1FE95DFC4F0190F081E02D7894B6
:102360000DC0E03129F0E13129F0E0E0F2E006C0F3
:1023700082E101C083E10E944B2BFC01CF01089553
:102380008CE060E00E947C2A8BE061E00E947C2A65
:102390008DE061E00E947C2A82E060E00E947C2A5D
:1023A00084E061E00E947C2A0895EF92FF920F93EF
:1023B0001F93009771F19C0140E050E068E478EED3
:1023C00081E090E00E94E62FC901DA017C018D01D5
:1023D00083E161E00E94E82A8FEFE816F10401052D
:1023E000110539F030F0FFEFEF2EF12C012D112DFA
:1023F0000AC0E114F1040105110529F4E1E0EE2E13
:10240000F12C012D112DE092B3008091B00080617C
:1024100007C083E160E00E94E82A8091B0008F7ECF
:102420008093B0001F910F91FF90EF900895A0E26C
:10243000B0E0EDE1F2E10C9409308CE00E94BA0AC0
:10244000882389F587E396E063E171E00E94462DD9
:102450005E9A409A80E00E94A00B0E947F0C5E98DA
:10246000409821C087E396E00E94C52E482F8091B6
:10247000BF04882321F0842F0E94900D14C0809106
:102480002A05E82FF0E031969F012F7130703197C7
:102490008091290590E02817390729F0E050FB4F7B
:1024A000408320932A0587E396E00E948B2E892B98
:1024B000C9F680919A03843009F08EC00E94F729F2
:1024C0006093AE047093AF048093B0049093B10412
:1024D000611571058105910561F481E090E0A0E04E
:1024E000B0E08093AE049093AF04A093B004B09397
:1024F000B1048091BA049091BB0481609093BB04B5
:102500008093BA0483E080939A038FE70E94960A2F
:1025100007EF14E00E94AA0AF80181938F01F5E009
:1025200000301F07B9F74091E2048091F704282F8B
:1025300030E0842F90E08227932786FF40C080E41C
:1025400048274093E204C90188739070C89709F541
:1025500010E014C01F5F8091F803E12FF0E084FFCA
:1025600006C0E950FB4F80810E94A20C07C0E950D1
:10257000FB4F87E396E060810E94FE2E212F30E022
:102580008091F70490E0877090708217930714F79A
:1025900016C02F733070232B91F48091F804809330
:1025A000B2048091F9048093B4048091FA0480937A
:1025B000B5048091FD048093BC041092BD04809109
:1025C0002B05813019F482E080932B0580912B0537
:1025D000833011F410922B050E94F7295B016C01E6
:1025E0008091B6049091B704A091B804B091B90459
:1025F0000097A105B105C9F086017501E81AF90A2D
:102600000A0B1B0BD801C701885B9B40A040B04060
:1026100060F00E94E10A8093B3041092B604109215
:10262000B7041092B8041092B90480ED93E00E94B0
:10263000F5082091AA043091AB044091AC0450916C
:10264000AD0486017501E21AF30A040B150BE616B8
:10265000F7060807190708F410C1A092AA04B0925F
:10266000AB04C092AC04D092AD04A8958091BE0496
:102670008830A0F08091A1039091A203A091A303C0
:10268000B091A4032CE1B695A795979587952A95C7
:10269000D1F70097A105B10509F08FC18091BE0463
:1026A0008F5F8093BE04E090AE04F090AF04009181
:1026B000B0041091B104E114F1040105110511F108
:1026C00080ED93E00E94F508AE18BF08C00AD10A59
:1026D0006A157B058C059D0588F48091A10384FD16
:1026E00004C080ED97E00E94D5111092AE041092C4
:1026F000AF041092B0041092B10404C080E090E0E6
:102700000E94D5119091E204907C9093E204009194
:102710002A05109129050117B1F180912B0582300E
:1027200091F590589093E20480ED93E00E94EB08BD
:10273000893010F048E002C0482F415030E013C00B
:102740003F5FA32FB0E0812F90E0FC01E050FB4FF2
:102750002081FD01EE51FB4F2083A05EBA4F2C93E8
:102760000196182F1F71341710F4101749F71093A2
:102770002905832F895C9091E204892B8093E204E0
:10278000309320051AC020912B052430D1F490916C
:102790002005E1E2F5E0A3EEB4E0292F30E02E0FB2
:1027A0003F1F02C081918D93E217F307D9F7995C1F
:1027B0008091E204982B9093E20483E080932B05B0
:1027C00038C08091A504823061F491609093E20456
:1027D0005E9A409A05EA13E07E010894E11CF11C20
:1027E00011C09093E2045E984098222319F481E08E
:1027F00080932B0580912B05833061F784E08093D3
:102800002B05E8CFF80181918F010E949F11F701FC
:10281000819391937F01F3E0053B1F0799F7809126
:10282000F8038770BE016F5F7F4F43EE54E00E9454
:102830007C095D9A419A8091A4040E94CB0A80EDA4
:1028400093E00E94EB08682F82EE94E00E948C0FC8
:10285000E091A404EF5FE093A404E83131F0F0E0EC
:10286000E053FC4F8785882341F41092A40405C0EF
:102870005E9A409A89E08093BE048091F803887143
:1028800071F180919A03823051F58091BA04909150
:10289000BB04880F991F9093BB048093BA0483E014
:1028A00080939A030E947F0C0E94F7296093B604DC
:1028B0007093B7048093B8049093B90461157105BF
:1028C0008105910561F481E090E0A0E0B0E08093A3
:1028D000B6049093B704A093B804B093B904809160
:1028E000F80384FF1EC08091BA049091BB048E7FD0
:1028F0000E943E0A182F8091B2046091BC040E948D
:102900007A0D082F8091B304612F0E947A0D282F31
:102910008091B4046091B504402F00919B030E9404
:102920000B115D9841988091A5048130D1F08130E0
:1029300020F0823009F047C034C082E10E941B2B96
:10294000892B09F040C081E08093A5040E94E92909
:102950006093A6047093A7048093A8049093A9049D
:1029600032C082E10E941B2B892B21F50E94E929AC
:102970002091A6043091A7044091A8045091A90485
:10298000621B730B840B950B695E73408040904013
:10299000D0F082E08093A50480ED97E00E94D511ED
:1029A00012C082E10E941B2B892B69F080E090E02D
:1029B0000E94D5111092A50406C08091BE048830F3
:1029C00009F058CF55CFA096EAE00C94253083E16A
:1029D00061E00E947C2A83E160E00E94E82A82E0B4
:1029E0008093B00085E08093B10083E061E00E94B5
:1029F0007C2A83E060E00E94E82A08951F93182F44
:102A00000E94F72960939F047093A0048093A1040F
:102A10009093A20410938D04112329F440E855E209
:102A200060E070E004C040E051EE60E070E087E3F9
:102A300096E00E94042E1F910895ACE1B0E0E3E21D
:102A4000F5E10C9409300E94F7297B018C0181E0AB
:102A50000E94A00B54E7A52E6E010894C11CD11C46
:102A600043E0B42EA982C60161E00E94C80FB09273
:102A70009A030E947F0C6AEF70E080E090E00E9471
:102A80001D2A80919A03833009F07DC087E396E088
:102A90000E948B2E892B09F076C00E94F7296E19AF
:102AA0007F09800B910B6058734C894C914008F062
:102AB0006AC0D8CF8FE70E94960A0E94AA0A84357E
:102AC00009F05CC089830E94AA0A182F00E01093C5
:102AD0008C0400938B040E94AA0A080F111D109306
:102AE0008C0400938B040E94AA0A80938A040E949B
:102AF000AA0A80938904813108F040C0FF2407C0EE
:102B00000E94AA0A07591B4FF8018083F3940F2DE6
:102B100010E08091890490E0880F991F0817190729
:102B200078F380E78983CE01019661E00E94C80FA7
:102B300083E080939A030E947F0C62E370E080E060
:102B400090E00E941D2A80919A038330A9F08FE7BC
:102B50000E94960A0E94AA0A803581F4898305EBB7
:102B600013E00E94AA0AF80181938F01F3E0003D6F
:102B70001F07B9F781E003C082E001C083E06C96D3
:102B8000EAE00C94253080919A03833009F092CFCB
:102B9000F3CF83E00E94BA0A8093F90384E00E9495
:102BA000BA0A8093FA0387E061E00E94C00A6AE0F3
:102BB00070E080E090E00E941D2A0E947F0C0000DF
:102BC00008950F931F93082F19C05E9A409A64E6E8
:102BD00070E080E090E00E941D2A5E98409864E6D4
:102BE00070E080E090E00E941D2A1F5F101768F3DC
:102BF0006CE271E080E090E00E941D2A10E0F6CFC8
:102C0000482F392F25E00DC0F999FECF1FBA842F28
:102C1000932F92BD81BD60BD0FB6F894FA9AF99AD0
:102C20000FBE215059F0F999FECF842F932F92BDFA
:102C300081BDF89A80B5681739F7089582E00E943F
:102C4000E1150895A0E0B0E0E8E2F6E10C9402306E
:102C5000482E562EEE24FF2488249924C0E0D0E08C
:102C6000CC24DD2416E4312E04C055245394CC2406
:102C7000DD24442069F480919B03839DE0011124AD
:102C8000BCE9EB2EB3E0FB2EA9E18A2E912C1DC0EE
:102C900021E0421671F480919B03839DE001112491
:102CA0006B96F0EDEF2EF3E0FF2EE9E28E2E912CE5
:102CB0000CC032E0431649F47BE9E72E73E0F72EAF
:102CC00061E0862E912CC8E1D1E03E016C0C7D1CA8
:102CD0001092340510923305E3011BC0552059F4BE
:102CE000F999FECFD2BDC1BDF89A80B5F701E00FCA
:102CF000F11F808307C0F701E00FF11FCE01608153
:102D00000E9400160E0D1F1DF80180810E943008E0
:102D100021969E012619022F10E008151905F0F2E0
:102D2000CE015520D9F4F999FECFD2BDC1BDF89A94
:102D300020B5F999FECF2196D2BDC1BD2197F89A51
:102D400080B590E0B22EAA248A299B2920913305D0
:102D5000309134052817390759F487CF21966091AF
:102D600034050E940016CE01609133050E940016C2
:102D700080E291E0C80ED91E91EEC91692E0D90604
:102D800008F477CF852DCDB7DEB7E1E10C941E3086
:102D900080E061E00E94221681E061E00E9422163C
:102DA000089580E060E00E942216882331F081E0DF
:102DB00060E00E942216882331F40E9492080E944B
:102DC0004D080E94C816089582E061E00E94221614
:102DD000089582E060E00E94221680919B03843077
:102DE00020F010929B030E94E41608951F93182F61
:102DF0000E94E91680919B03811731F0143020F472
:102E000010939B030E94E4161F910895109267048B
:102E100085E6E2E0F4E0DF011D928A95E9F7089586
:102E20001F93182F8F3711F08830E1F5E091670478
:102E3000EE2309F455C0E150E0936704F0E0EE5F43
:102E4000FB4F108287E396E06DE00E94FE2E10E0BB
:102E50000AC0E12FF0E0EE5FFB4F87E396E0608170
:102E60000E94FE2E1F5F80916704181790F387E37E
:102E700096E060E20E94FE2E87E396E06DE00E94FD
:102E8000FE2E10E00AC0E12FF0E0EE5FFB4F87E37B
:102E900096E060810E94FE2E1F5F809167041817E4
:102EA00090F31CC08B3119F40E9406171FC08D309F
:102EB000E9F08A30D9F080916704843688F487E39A
:102EC00096E0612F0E94FE2E80916704E82FF0E0CB
:102ED000EE5FFB4F10838F5F8093670480E007C035
:102EE00087E396E067E00E94B22BF8CF81E01F9164
:102EF00008951F93CF93DF93CFEDD3E010E03BC055
:102F000087E396E062E271E00E94432D87E396E05A
:102F1000612F4AE050E00E94C02C87E396E06FE208
:102F200071E00E94432D699170E080E090E0209173
:102F3000DE0330E040E050E00E94922F20E137E2D3
:102F400040E050E00E94922FDC01CB014091D5037C
:102F50005091D6036091D7037091D803480F591F41
:102F60006A1F7B1F87E396E02AE030E00E94872CEF
:102F70001F5F183119F08881882311F6DF91CF91F6
:102F80001F910895EF92FF920F931F93882339F4B6
:102F900087E396E061E77AE00E94D02B3BC090E0A7
:102FA0000E94B20824E630E040E050E00E94C42FC6
:102FB000122F032FF42EE52E622F732F842F952FBF
:102FC0002AE030E040E050E00E94C42F87E396E022
:102FD000BA01A9012AE030E00E94782C87E396E04C
:102FE0006EE20E94B22B612F702F8F2D9E2D2AE052
:102FF00030E040E050E00E94C42FAB01BC0187E309
:1030000096E02AE030E00E94782C87E396E063E7C0
:103010000E94E42B1F910F91FF90EF900895FF9273
:103020000F931F93CF93DF9387E396E067E67AE0F1
:103030000E94912B8091B503813041F487E396E0A3
:103040006EE47AE00E94D02BFF246DC0823029F418
:1030500087E396E067E37AE0F5CF843029F487E3ED
:1030600096E063E27AE0EECF853071F787E396E091
:1030700068E17AE0E7CFCF2DD0E0C930D1051CF070
:103080006F2D685C02C06F2D6F5C87E396E00E9435
:10309000B22B87E396E060E17AE00E94912BBE01BB
:1030A0006F5F7F4F87E396E04AE050E00E941C2D5F
:1030B00087E396E065E07AE00E94912B8E010B5445
:1030C0001C4FD8011196EC91E032F8F487E396E0BA
:1030D00068EF79E00E94912BF8018181803130F016
:1030E00087E396E063E371E00E94432DCB54DC4F0D
:1030F000698170E06F7070706F5F7F4F87E396E05B
:103100004AE050E00E942F2D0DC0F0E0EF70F0700B
:10311000EE0FFF1FE75BFC4F6081718187E396E054
:103120000E94462DF39480918A04F81608F4A3CFE8
:1031300087E396E06DED79E00E94912B8091CD03BD
:103140000E94C21787E396E062EC79E00E94912B1F
:103150008091CE030E94C21787E396E067EA79E088
:103160000E94912B8091CF030E94C21787E396E0C3
:103170006CE879E00E94912B4091C5035091C60301
:103180006091C7037091C803411551056105710530
:1031900039F187E396E02AE030E00E94872C87E34C
:1031A00096E069E579E00E94912B8091C9030E9425
:1031B000E508AB01BC0187E396E02AE030E00E941D
:1031C000872C87E396E065E379E00E94912B87E303
:1031D00096E06091CA034AE050E00E94D22C06C0FB
:1031E00087E396E06CE279E00E94D02B87E396E0DB
:1031F0006FE079E00E94912B6091CB037091CC033A
:1032000087E396E04AE050E00E94AC2C87E396E02A
:1032100062EF78E00E94912B6091C403603450F417
:1032200070E06F5F7F4F87E396E04AE050E00E94D6
:103230002F2D06C087E396E069EE78E00E94D02B40
:1032400087E396E06CEC78E00E94912B8091C303B9
:1032500080FD03C065E371E002C069E371E087E3CC
:1032600096E00E94462D87E396E06FEA78E00E94A0
:10327000912B8091C30382700E94840D87E396E0B6
:1032800060E978E00E94912B8091C30384700E94D2
:10329000840D87E396E061E778E00E94912B8091AE
:1032A000C30388700E94840DCDB7DEB7E5E00C94AF
:1032B0002A301F93CF93DF9387E396E06BEB7BE09D
:1032C0000E94912B4091D5035091D6036091D70372
:1032D0007091D80387E396E02AE030E00E94872CC3
:1032E00087E396E065EA7BE00E94912B4091D90349
:1032F0005091DA036091DB037091DC0387E396E081
:1033000020E130E00E94872C87E396E06FE87BE0C5
:103310000E94912B87E396E06091DD034AE050E044
:103320000E94D22C87E396E069E77BE00E94912B14
:1033300087E396E06091DE034AE050E00E94D22CE1
:1033400087E396E063E67BE00E94912BCFEDD3E02C
:1033500010E012C0112331F087E396E06DE371E0D5
:103360000E94432D87E396E069914AE050E00E9475
:10337000C02C1F5F183119F08881882359F787E323
:1033800096E00E94BA2B87E396E06DE47BE00E9412
:10339000912B87E396E06091F7034AE050E00E94AA
:1033A000D22C87E396E068E37BE00E94912BE091CA
:1033B000F803F0E0E770F070EE0FFF1FE759FC4FE5
:1033C0006081718187E396E00E94462D87E396E055
:1033D00063E27BE00E94912B8091F80390E088717A
:1033E00090708830910589F0893091051CF4892B03
:1033F00039F01BC08031910569F04897B1F40FC0D6
:1034000087E396E06AE17BE00EC087E396E06EE03A
:103410007BE009C087E396E068E07BE004C087E3D7
:1034200096E06EEF7AE00E94D02B87E396E06AEE9A
:103430007AE00E94912B4091D1035091D203609188
:10344000D3037091D40387E396E02AE030E00E9432
:10345000872C87E396E061ED7AE00E94912B8091C2
:10346000A10380710E94840D87E396E068EB7AE007
:103470000E94912B8091A10380740E94840D87E3A8
:1034800096E06FE97AE00E94912B8091A10380720F
:103490000E94840D87E396E062E87AE00E94912B17
:1034A00080ED93E00E94F508AB01BC0187E396E054
:1034B0002AE030E00E94782C87E396E06DE77AE01E
:1034C0000E94912B80ED93E00E94F5089B01AC01D6
:1034D00060E472E48FE090E00E94C42F87E396E0FE
:1034E000BA01A9012AE030E00E94782C87E396E037
:1034F0006AE77AE00E94D02BDF91CF911F91089567
:10350000EF92FF920F931F937C0107E316E0C8012F
:103510006F2D70E04AE050E00E949B2CC8016EE2E3
:103520000E94B22BB70124E0769567952A95E1F7C2
:103530006F707070C8014AE050E00E949B2CC80177
:103540006EE20E94B22B8FE0E822FF24C801B7018F
:103550004AE050E00E949B2C1F910F91FF90EF904A
:1035600008950F931F93CF93DF93209101042F3F72
:10357000A9F587E396E061EF75E00E94912B81E762
:1035800093E00E94801A87E396E060ED75E00E9468
:10359000912B80918B0490918C040E94801A87E378
:1035A00096E06DE975E00E94D02B87E396E06AE72C
:1035B00075E00E94D02B87E396E062E675E00E94FA
:1035C000D02B87E396E06DE375E00E94D02B87E374
:1035D00096E00E94BA2B0E940F1869C012160CF0D8
:1035E00066C0332727FD309580918A0490E08217CA
:1035F00093070CF45CC087E396E068E275E00E94F4
:10360000912B60910104772767FD709587E396E021
:103610004AE050E00E942F2D87E396E06DEF74E0C2
:103620000E94912B10E008E23AC0C12FD0E0CC0FED
:10363000DD1FC759DB4F288130E0809101049927B5
:1036400087FD909501972817390741F587E396E0A4
:103650006FE371E00E94432D87E396E0602F4AE01C
:1036600050E00E94C02C87E396E063E471E00E9482
:10367000432DE981F0E0EF70F070EE0FFF1FE75B84
:10368000FC4F6081718187E396E00E94432D87E3C0
:1036900096E067E471E00E94432D0F5F1F5F809109
:1036A0008904181710F287E396E00E94BA2BDF9185
:1036B000CF911F910F910895ACE1B0E0E2E6FBE1FC
:1036C0000C940B30282F809101048F3F09F042C1E8
:1036D000822F90E0FC013A97EF36F10508F033C1F4
:1036E000EC5CFF4F0C94383087E396E069E471E0BE
:1036F000AEC087E396E069E471E00E94462D1CC1EC
:1037000087E396E065E571E00E94462D85E78983B1
:10371000DE011296E5EBF3E08BE101900D92815012
:10372000E1F7CE0101966CE10E94C80F0E947F0C68
:1037300083E080939A0368EC70E080E090E00E9460
:103740001D2A80919A03843009F0FDC08FE70E9402
:10375000960A0E94AA0A8983853509F0F4C087E396
:1037600096E06FED74E00E94D02B87E396E061EC69
:1037700074E00E94D02B87E396E063EA74E0ACC06B
:1037800087E396E06DE671E00E94462D89E6898325
:10379000CE01019661E00E94C80F0E947F0C83E079
:1037A00080939A0368EC70E080E090E00E941D2A0C
:1037B00080919A03843009F0C6C08FE70E94960A70
:1037C0000E94AA0A89838E010E5F1F4FBDE1EB2E76
:1037D000F12CEC0EFD1E0E94AA0AD8018D938D01DA
:1037E000AE15BF05C1F7A5EBB3E0FE0132968BE144
:1037F00001900D928150E1F78981893409F0A3C0CD
:1038000087E396E065E874E00E94D02B87E396E0BA
:1038100067E674E00E94D02B87E396E069E474E0E9
:103820005BC087E396E067E871E00E94462D8EEF6B
:103830008093010488C020522750922F905380918A
:103840008A04891738F487E396E066E971E00E94FC
:10385000462D79C0909301046FC084E180930104E8
:1038600087E396E062E174E037C085E1809301046C
:1038700087E396E06BED73E02FC086E1809301044F
:1038800087E396E064EA73E027C087E18093010450
:1038900087E396E06AE573E01FC088E18093010446
:1038A00087E396E069E473E017C089E1809301043F
:1038B00087E396E065E373E00FC08AE1809301043B
:1038C00087E396E060E273E007C08BE18093010438
:1038D00087E396E068EF72E00E94D02B34C087E364
:1038E00096E06EED72E00E94D02B8091C30391E0D0
:1038F0001DC087E396E068EC72E00E94D02B8091B7
:10390000C30392E013C087E396E063EB72E00E948A
:10391000D02B8091C30394E009C087E396E068E967
:1039200072E00E94D02B8091C30398E08927809396
:10393000C3038FEF809301040E94B11A04C087E390
:1039400096E00E94C52E87E396E00E948B2E892B7D
:10395000B1F762C1822F0E941017882309F45CC15D
:1039600080916704882321F48FEF809301044CC178
:1039700082E094E060E070E040E050E00E94A20647
:103980009B01AC0160910104862F992787FD9095DA
:10399000A92FB92FFC013197EB31F10508F024C1B3
:1039A000ED55FF4F0C943830E62FFF27E7FDF095DB
:1039B00080918A0490E08E179F070CF415C1DA01FC
:1039C000C9010197A109B1098097A105B10548F086
:1039D000A8E2FA2E00E010E06F010894C108D108B7
:1039E00025C0EB54FC4F822F81508083E5C0612FAE
:1039F00070E0660F771F67597B4FFB01808190E075
:103A00008C159D0591F48F2D90E0A0E0B0E0821719
:103A10009307A407B50741F4F601EB54FC4FDB0113
:103A200011968C91818301E0F3941F5F809189044A
:103A30001817E8F2BFC02F3F31054105510511F0BD
:103A400008F0D2C02093CD03B7C02F3F3105410508
:103A5000510511F008F0C8C02093CE03ADC02F3F30
:103A600031054105510511F008F0BEC02093CF0388
:103A7000A3C0809102048062803719F583E094E04E
:103A800060E070E040E050E00E94A2069B01AC01C3
:103A9000DC01CB010197A109B1090897A105B10586
:103AA00008F0B5C0CA01B90124ED30E340E050E0B0
:103AB0000E94922F9B01AC012A5E3C4A4A46554E19
:103AC00024C0863611F583E094E060E070E040E0C9
:103AD00050E00E94A2069B01AC01DC01CB010197E2
:103AE000A109B1090797A105B10508F090C0CA0165
:103AF000B90128EA31E640E050E00E94922F9B0194
:103B0000AC01245E3C434E46544E2115310541051F
:103B1000510561F0DA01C901805C9D49A845B543B2
:103B200081509A45A246B24008F05EC02093C5037A
:103B30003093C6034093C7035093C8033DC02F3F43
:103B400031054105510511F008F04EC02093C9031D
:103B500033C0DA01C9010197A109B1098F3F91056D
:103B6000A105B10508F040C02093CA0325C0DA01C1
:103B7000C901845C9940A040B0408D549D41A04053
:103B8000B04030F43093CC032093CB0301E001C06C
:103B900000E0211531054105510511F48FEF07C0F3
:103BA000213431054105510528F4822F815080933D
:103BB000C40302C00023C1F0809168048823D1F4BB
:103BC0008091D9039091DA03A091DB03B091DC03DB
:103BD0000196A11DB11D8093D9039093DA03A093A0
:103BE000DB03B093DC0306C087E396E068EA71E08C
:103BF0000E94462D0E9406178FEF8093010487E3F1
:103C000096E06AE00E94E42B0E94B11A05C021E010
:103C100030E040E050E07ECF6C96E8E00C94273036
:103C200087E396E06CE472E00E94D02B87E396E095
:103C300064E372E00E94D02B87E396E00E948B2E13
:103C4000892B31F087E396E00E94C52E0E945C1B11
:103C50000E941D15823019F0833069F405C087E396
:103C600096E066E172E004C087E396E06FEF71E0F2
:103C70000E94D02B08958FEF809301041092680466
:103C80000E94B11A0CC087E396E00E948B2E892B0C
:103C900031F087E396E00E94C52E0E945C1B809164
:103CA00001048E3F81F7089580910104992787FDD3
:103CB0009095A92FB92FFC013196EB30F10508F052
:103CC00074C0E254FF4F0C94383087E396E064E60A
:103CD00078E00E94D02B81E793E00E94801A87E36E
:103CE00096E06CE478E00E94D02B87E396E067E2F0
:103CF00078E00E94D02B87E396E06DEF77E00E949A
:103D0000D02B87E396E06CED77E00E94D02B87E321
:103D100096E06FEA77E00E94D02B87E396E069E8AF
:103D200077E00E94D02B87E396E065E677E00E947B
:103D3000D02B87E396E06EE377E00E94D02B87E3F9
:103D400096E00E94BA2B0E9459192FC087E396E093
:103D500061E277E028C087E396E06CEF76E023C06D
:103D600087E396E067EE76E01EC087E396E068ECB6
:103D700076E019C087E396E064E876E014C087E354
:103D800096E06FE676E00FC087E396E06AE576E0BE
:103D90000E94D02B87E396E064E176E004C087E3DD
:103DA00096E06EEF75E00E94D02B6AE070E080E054
:103DB00090E00E941D2A04C087E396E00E94C52E71
:103DC00087E396E00E948B2E892BB1F70895A2E23B
:103DD000B0E0EDEEFEE10C9401308E010F5F1F4F5D
:103DE00080E1D8011D928A95E9F787E396E066ECB9
:103DF00071E00E94462D0E94C91520EC3DE948E57E
:103E000055E32F8F38A349A35AA380EC97EFAAEB71
:103E1000B7E38B8F9C8FAD8FBE8F24EF31E040E0F6
:103E200050E02F8B388F498F5A8F30E5C32E33ECFB
:103E3000D32EE12CF12C20EC422E2DE9522E28E538
:103E4000622E25E3722E88249924540133241E8A7D
:103E50001D8A198A1A8A1B8A1C8AFFC087E396E08A
:103E60000E94C52E8434B9F0853430F48332B9F120
:103E70008C3209F0CCC044C0833509F0C8C02F8D06
:103E800038A149A15AA1C901DA012C013D018824B8
:103E900099245401E2C087E396E064E40E94B22BC7
:103EA00087E396E040EC5DE968E575E32AE030E001
:103EB0000E94E62C87E396E06CE20E94B22B87E337
:103EC00096E040EC57EF6AEB77E32AE030E00E949F
:103ED000E62C87E396E06CE20E94E42BBEC01982D8
:103EE0001A821B821C821D821E821F8218861986DE
:103EF0001A861B861C861D861E861F86188A3AC057
:103F0000339434E0331609F0A8C069817A818B813B
:103F10009C8128EE33E040E050E00E94922F6F8FAA
:103F200078A389A39AA36D817E818F8198850E9451
:103F3000922F6B8F7C8F8D8F9E8F89859A85AB8515
:103F4000BC858F8B988FA98FBA8F6D857E858F8565
:103F500098890E94922F6B017C0190E2C9169EE421
:103F6000D90690E0E90690E0F90630F48CE162E3CE
:103F70000E94C00A332471C0A0E3CA16A5E7DA067E
:103F8000A0E0EA06A0E0FA0618F48CE162E2F0CFC5
:103F9000B0E4CB16BCE9DB06B0E0EB06B0E0FB0614
:103FA00018F48CE166E2E4CFE0E5CE16E3ECDE0641
:103FB000E0E0EE06E0E0FE0618F48CE162E1D8CF26
:103FC000F0E6CF16FAEEDF06F0E0EF06F0E0FF06CF
:103FD00018F48CE165E1CCCF20E7C21621E1D206CE
:103FE00021E0E20620E0F20618F48CE161E0C0CFA7
:103FF00030EAC31636E8D30631E0E30630E0F306D4
:1040000018F48CE163E0B4CF8CE165E0B1CF90EDC2
:10401000292E280E49E0421500F1032D10E0000F73
:10402000111F000F111F81E090E08C0F9D1F080FE2
:10403000191FD8016D917D918D919C912AE030E0FE
:1040400040E050E00E94922F620D711D811D911D74
:10405000F801608371838283938387E396E00E94F3
:104060008B2E892B09F0FACE81149104A104B1049E
:1040700089F4C301B2010E94360B61E070E080E078
:1040800090E00E941D2AFFEFFE8B1D8A198A1A8A72
:104090001B8A1C8A2F89388D498D5A8D821693066A
:1040A000A406B506E0F40E94E10A29893A894B8901
:1040B0005C89280F311D411D511D298B3A8B4B8B7B
:1040C0005C8B3D89381708F48D8B4E89841708F472
:1040D0008E8B0894811C911CA11CB11C56C0C3017D
:1040E000B20128EE33E040E050E00E94C42F87E3A5
:1040F00096E0BA01A9012AE030E00E94782C87E31B
:1041000096E06CE20E94B22B87E396E06D894AE06C
:1041100050E00E94C02C87E396E06CE20E94B22B34
:1041200069897A898B899C89A50194010E94C42F91
:1041300087E396E0BA01A9012AE030E00E94782CDA
:1041400087E396E06CE20E94B22B87E396E06E89EB
:104150004AE050E00E94C02C87E396E06CE20E94A7
:10416000E42B4C0C5D1C6E1C7F1C8B8D9C8DAD8DCF
:10417000BE8D84159505A605B70520F44F8C58A073
:1041800069A07AA08824992454012F8D38A149A1CF
:104190005AA1285E33404040504009F05ECFA296BD
:1041A000E2E10C941D30AAE5B0E0E9EDF0E20C94F8
:1041B0000D308B017A018B3009F426C18C3040F52B
:1041C000853009F484C0863080F4823009F459C007
:1041D000833020F4813009F050C242C0833009F4AA
:1041E00061C0843009F049C265C0883009F49DC0BF
:1041F000893038F4863009F486C0873009F03DC232
:104200008CC0893009F499C08A3009F036C2C9C01F
:10421000893609F482C18A3680F4863609F42DC1C4
:10422000873620F4853609F028C20EC1873609F496
:104230003DC1883609F021C241C18C3609F4C4C1A0
:104240008D3638F48A3609F473C18B3609F015C2FD
:10425000AFC18D3609F4ECC1873C09F00EC200C233
:1042600081E069E270E00E94801100ED13E0F80146
:1042700081918F010E946911F3E0093F1F07B9F78F
:1042800004C282E06BE170E00E94801105EB13E054
:10429000F80181918F010E946911F3E0003D1F0731
:1042A000B9F7F3C183E061E070E00E9480110E94E1
:1042B0001D15E9C184E061E070E00E94801181E099
:1042C0000E9469110E9462110E94E71EE0C1609184
:1042D000890470E0660F771F85E00E94801100E07E
:1042E00010E008C0F801E759FB4F80810E94691176
:1042F0000F5F1F4F8091890490E0880F991F081766
:10430000190780F3C2C186E062E070E00E9480116C
:1043100081E793E00E947711B8C187E061E070E027
:104320000E94801180918A04AEC188E061E070E053
:104330000E94801180919B03A6C186E68983CE01ED
:10434000019661E00E94C80F0E947F0C83E0809379
:104350009A0368EC70E080E090E00E941D2A809152
:104360009A038430E1F48FE70E94960A0E94AA0A19
:104370008983863471F489E060E270E00E948011E4
:1043800010E00E94AA0A0E9469111F5F1032C9F74B
:104390007CC189E061E070E00E948011C7C089E0C3
:1043A0006DC18AE069E170E00E94801182E0809333
:1043B0009C038091A105882351F08091A1039091E5
:1043C000A203A091A303B091A403806809C08091C7
:1043D000A1039091A203A091A303B091A4038F77AE
:1043E0008093A1039093A203A093A303B093A4038B
:1043F0000CE913E0F80181918F010E946911F3E04B
:10440000053B1F07B9F741C18BE061E270E00E94F4
:1044100080118091BE048F3F39F08091BE048F5F80
:104420008093BE04815002C08091BE040E94691135
:1044300010E0812F0E949F110E94190A0E9477119B
:104440001F5F1031B1F721C185E661E070E00E9485
:1044500080110932110509F015C120E030E0F901A1
:10446000E053FC4FD701A20FB31F8C9180832F5FC5
:104470003F4F2932310599F759C086E661E070E077
:104480000E9480110B31110509F0FCC020E030E0E2
:10449000F901EB54FC4FD701A20FB31F8C9180831D
:1044A0002F5F3F4F2B31310599F740C087E661E020
:1044B00070E00E9480110E94C81638C088E661E052
:1044C00070E00E94801185E78A83DE011396E5EB98
:1044D000F3E08BE101900D928150E1F7CE0102965D
:1044E0006CE10E94C80F0E947F0C83E080939A03C6
:1044F00060E273E080E090E00E941D2A80919A03C0
:10450000843009F0BFC08FE70E94960A0E94AA0A71
:104510008A83853509F0B6C009C089E661E070E09C
:104520000E9480110E944D080E94920881E0ABC059
:104530008AE661E070E00E94801189E68E8FCE01EC
:104540004E9661E00E94C80F0E947F0C83E080932A
:104550009A0360E273E080E090E00E941D2A80915F
:104560009A03843009F08EC08FE70E94960A0E9459
:10457000AA0A8E8F8E01015E1F4F4AE3E42EF12CB2
:10458000EC0EFD1E0E94AA0AF80181938F01EE1520
:10459000FF05C1F7A5EBB3E0FE017F968BE101902B
:1045A0000D928150E1F78E8D893409F06BC0BECF3A
:1045B0008BE661E070E00E948011F70180810E942B
:1045C000F6160E94D116B2CF8CE661E070E00E9430
:1045D00080110032110571F487E68AAFDE01DB96A7
:1045E000F70180E201900D928150E1F7CE01CA9669
:1045F00061E205C087E48AAFCE01CA9661E00E94FD
:10460000C80F0E947F0C83E080939A036CE474E0EF
:1046100080E090E00E941D2A80919A03843091F5F9
:104620008FE70E94960A0E94AA0A873459F57ECF26
:104630008DE661E070E00E9480110931110511F5ED
:1046400020E030E0F901E456FC4FD701A20FB31F80
:104650008C9180832F5F3F4F2931310599F766CFC9
:1046600087EC61E070E00E94801181E00E94691196
:104670000E9462111092FF030AC08AEC61E070E0B0
:104680000E94801180E00E9469110E946211C65A46
:10469000DF4FE6E00C942930A0E0B0E0E2E5F3E281
:1046A0000C94093084E0A82E06E0B02E15E0C12E4F
:1046B00005E315E0B4E6DB2EA2E0EA2EF3E0FF2EE0
:1046C000A1C087E396E00E94C52E982F8093A00595
:1046D00080919F05833021F1843028F4813099F056
:1046E0008230B8F409C0853009F448C0853020F123
:1046F000863009F087C05FC0953B09F083C081E038
:1047000080939F057FC0923609F07AC0E0929F05A2
:1047100079C090939E0590939D05F0929F0572C07D
:1047200090939B0510929C0580919D05892780930D
:104730009D05A0929F0566C0D92FC0E020919B05E2
:1047400030919C052C2B3D2B30939C0520939B0591
:1047500080919D05892780939D05C0929F052536F0
:10476000310508F44FC08CEC61E070E00E948011CC
:1047700081E00E9469110E94621142C02091990556
:1047800030919A05F901EB5CFA4F908380919D0579
:10479000892780939D052F5F3F4F30939A05209383
:1047A000990580919B0590919C052817390750F138
:1047B000B0929F0527C080919D05891759F460919B
:1047C000990570919A0580919E0545E355E00E94F8
:1047D000D3200DC08BEC62E070E00E9480118091CC
:1047E0009E050E946911809100040E946911F801E0
:1047F0008D2D11928A95E9F710929A0510929905DC
:1048000010929F0587E396E00E948B2E892B09F07A
:1048100058CFCDB7DEB7EAE00C94253081E0809325
:10482000FF0308C087E396E00E948B2E892B11F0CE
:104830000E944C238091FF038823A1F70895A0E0F4
:10484000B0E0E5E2F4E20C940C300E94F729611527
:10485000710581059105C9F30E9499061092D9034B
:104860001092DA031092DB031092DC03DD24E09057
:10487000D903F090DA030091DB031091DC03102FD1
:104880000F2DFE2CEE240E9494062FEF30E040E026
:1048900050E00E94E62FE60EF71E081F191FE09257
:1048A000D903F092DA030093DB031093DC03D39473
:1048B00044E0D416E1F6CFEDD3E000E010E090E163
:1048C000E92E97E2F92E4EC00F5F19F40E944D08B1
:1048D0004DC00E94940622E330E040E050E00E9488
:1048E000E62F6F5FEFEDF3E090E004C08191861753
:1048F00059F39F5F9117D0F38091DE0390E08E9D76
:1049000090018F9D300D9E9D300D1124862F90E0DB
:10491000AC01249FC001259F900D349F900D112460
:10492000AA2797FDA095BA2F2091D5033091D603E1
:104930004091D7035091D803820F931FA41FB51F36
:1049400020919D0330919E0340919F035091A003BD
:10495000281739074A075B0708F4B6CF69931F5F2A
:10496000183121F08881882309F0AECFCDB7DEB7AA
:10497000E7E00C9428301F93109101041F3F09F0C9
:10498000F1C0893409F467C08A3428F5883309F402
:1049900079C0893368F4803309F486C0813308F024
:1049A0006FC08B3109F44DC0813209F0D5C03DC0D4
:1049B000813409F49AC0823438F4893309F472C01E
:1049C000803409F0C9C031C0823409F4A1C08634F2
:1049D00009F0C2C052C0823609F49AC0833690F4FE
:1049E000883579F1893538F4823509F43FC083354B
:1049F00009F0B2C01FC08A3509F4A9C0813609F098
:104A0000ABC073C0823791F1833730F48636A9F199
:104A1000893609F0A1C01FC0883799F08A3709F498
:104A200096C0833709F098C005C087E396E069E433
:104A300071E019C00E94C81687E396E063ED71E04B
:104A400006C00E94D11687E396E06DEE71E00E94E9
:104A5000462D8EEF7FC00E944D080E94920887E38A
:104A600096E06CE072E00E94462D76C00E941F2402
:104A700087E396E065E272E0F6CF0E9479176CC09A
:104A8000805368C087E396E06CEE71E00E94D02B03
:104A90009091F803892F885F8871977E892B809386
:104AA000F80320C089E056C087E396E069ED71E025
:104AB0000E94D02B8091A1039091A203A091A30307
:104AC000B091A40320E130E040E050E0822793273A
:104AD000A427B5278093A1039093A203A093A303D7
:104AE000B093A4031093010437C087E396E063EC0E
:104AF00071E00E94D02B8091A1039091A203A0911C
:104B0000A303B091A40320E430E040E050E012C0E1
:104B100087E396E062EB71E00E94D02B8091A103C5
:104B20009091A203A091A303B091A40320E230E0EE
:104B300040E050E082279327A427B5278093A10364
:104B40009093A203A093A303B093A40302C00E9476
:104B5000101E8FEF80930104809101048E3F09F4B1
:104B6000DDC0D4C00E941017882309F4D7C08091FB
:104B70006704882321F48FEF80930104C7C082E08B
:104B800094E060E070E040E050E00E94A2069B01EB
:104B9000AC0180910104992787FD9095A92FB92F29
:104BA000FC013197E930F10508F08CC0E753FF4F65
:104BB0000C943830DA01C901815C9D49A845B543A0
:104BC0008F5F9945A246B24008F07CC02093D50380
:104BD0003093D6034093D7035093D8039AC02093C1
:104BE000D9033093DA034093DB035093DC0381E075
:104BF000809368048EC0283031054105510508F0C6
:104C000061C02093DD0385C0DA01C9010197A109C4
:104C1000B1090A97A105B10508F054C02093DE033D
:104C200078C082E094E06DE371E00E94BE0710E07E
:104C30000EC0183130F4E12FF0E0E053FC4F8787CD
:104C40001F5F80E090E06DE371E00E94BE07009777
:104C500059F00E94A007009761F706C0E12FF0E02D
:104C6000E053FC4F17861F5F1831C0F352C0253048
:104C700031054105510530F52093F7034AC0DA01AB
:104C8000C9010197A109B1090697A105B105D0F4A1
:104C90008091F803887F822B8093F8033AC0DA0171
:104CA000C9010197A109B1098050924CA140B040BF
:104CB00048F42093D1033093D2034093D30350930D
:104CC000D40327C087E396E068EA71E00E94462D8E
:104CD00013C08091D9039091DA03A091DB03B091C6
:104CE000DC030196A11DB11D8093D9039093DA03D3
:104CF000A093DB03B093DC030E9406178FEF809331
:104D0000010487E396E06AE00E94E42B0E94541EAF
:104D100005C0809168048823E1F2EECF1F910895C9
:104D20008FEF80930104109268040E94541E0CC0FF
:104D300087E396E00E948B2E892B31F087E396E083
:104D40000E94C52E0E94BB24809101048E3F81F7F2
:104D50006AE070E080E090E00E941D2A04C087E3D2
:104D600096E00E94C52E87E396E00E948B2E892B49
:104D7000B1F70895AAE2B0E0E0ECF6E20C94063058
:104D80000E94E9297B018C0181E00E94A00B04C0F4
:104D900087E396E00E94C52E87E396E00E948B2E63
:104DA000892BB1F75E984098DD24D39452E6752E96
:104DB00042E0842E912C8C0E9D1E5E010894A11C55
:104DC000B11C33E0C32E0E94E92920E030E06E19C7
:104DD0007F09800B910B693C71058105910510F0ED
:104DE00021E030E08D2D90E028233923232BA9F1F9
:104DF0000E94E9297B018C015D9A419A80ED97E040
:104E00000E94D5117982D401E0EDF3E089E20190AE
:104E10000D928150E1F7C5016AE20E94C80F5D98CA
:104E2000419880E090E00E94D511C0929A030E94C0
:104E30007F0C62E370E080E090E00E941D2A809188
:104E40009A03843051F4C0929A038FE70E94960A25
:104E50000E94AA0A823409F4DD2482E10E941B2BFD
:104E6000892B69F5DD24D3942AC05E9A409A5D9A15
:104E7000419A87E396E00E94C52E8D30910569F036
:104E80008E3091051CF40A97B1F407C08332910566
:104E900069F08234910579F40CC087E396E064EA06
:104EA00071E00E94D02B0E94902605C00E94E71E50
:104EB00002C00E940E245E9840985D98419887E356
:104EC00096E00E948B2E892B09F47DCFCECF8F9256
:104ED0009F92AF92BF92CF92DF92EF92FF920F9389
:104EE0001F9382E10E941B2B892B09F083C068EC81
:104EF00070E080E090E00E941D2A80E090E00E9437
:104F0000D5110E94E9295B016C0160ECE62E62E19B
:104F1000F62E012D112DEA0CFB1C0C1D1D1D06C0CB
:104F200082E10E941B2B892B09F062C00E94E929B3
:104F30006E157F058007910798F382E10E941B2B75
:104F4000892B09F055C080ED97E00E94D5110E9491
:104F5000E9297B018C0199249394882488E496E2C2
:104F6000A0E0B0E0A80EB91ECA1EDB1E29C0AE1418
:104F7000BF04C006D10638F480ED97E00E94D51139
:104F8000882483941DC00E94E9296E197F09800B33
:104F9000910B693C71058105910590F00E94E9290A
:104FA0007B018C0180E0992009F481E0982E882310
:104FB00019F480E090E002C080ED97E00E94D511E6
:104FC00082E10E941B2B892B91F280E090E00E94ED
:104FD000D511882049F080919B038F5F83700E94D8
:104FE000F6160E94D11606C00E941F240E94C81601
:104FF0000E94BA261F910F91FF90EF90DF90CF9003
:10500000BF90AF909F908F90089580E06DEF77E014
:1050100042E050E00E9424290895EF92FF920F93FE
:105020001F9380E00E9419080E94C01186E061E091
:105030000E947C2A85E061E00E947C2A8EE061E08B
:105040000E947C2A8FE061E00E947C2A82E160E07D
:105050000E947C2A88E060E00E947C2A88E061E06F
:105060000E94E82A0E94E71487E396E040E052ECB1
:1050700061E070E00E94042E0E94E9160E94D116A1
:105080000E945F0D8FEF8093BE040E9405287894E4
:105090000E94E9297B018C018091BE048F3F09F0B9
:1050A000C8C00E94E9296E197F09800B910B605DD1
:1050B00077408040904008F0BCC0EECF87E396E098
:1050C0000E94C52E87E396E00E948B2E892BB1F7B4
:1050D00087E396E062E472E00E94432D81E793E06B
:1050E0000E94801A87E396E069E572E00E94432DF2
:1050F00087E396E065E070E04AE050E00E942F2DE3
:1051000062E370E080E090E00E941D2A87E396E071
:105110000E948B2E04970CF187E396E00E94C52E27
:1051200082349105D1F487E396E00E94C52E8E3437
:10513000910599F487E396E00E94C52E8434910589
:1051400061F487E396E00E94C52E819731F480E0F8
:1051500090E00E94D5110E94BA264091D10350914F
:10516000D2036091D3037091D403DB01CA0101978C
:10517000A109B1090497A105B10568F44093BF04E2
:10518000433029F040E052EC61E070E004C040EAB6
:1051900056E861E070E087E396E00E94042E0E94EA
:1051A00067275E98409880E090E00E94D5110E94A9
:1051B0005F0D80E00E94A00B8091A4040E94CB0AA6
:1051C0000E947F0C1092290510922A0510922B053F
:1051D00010E015C062E370E080E090E00E941D2ABC
:1051E00080ED97E00E94D51162E370E080E090E0EE
:1051F0000E941D2A80E090E00E94D5111F5F8091DF
:105200009B03811738F78091F80390E084FF09C071
:1052100020E088719070489709F421E0822F0E9465
:10522000FE148FE00E9419081F910F91FF90EF90DC
:10523000089580ED97E00E94D51182E161E00E941F
:10524000E82A5E9A409A3ECF823000F5E82FF0E0DF
:10525000EE0FFF1FEE55FA4F71836083882319F01C
:105260008130A1F408C0809169008C7F842B8093E9
:105270006900E89A089580916900440F551F440F12
:10528000551F837F842B80936900E99A08951F92AC
:105290000F920FB60F9211242F933F934F935F936A
:1052A0006F937F938F939F93AF93BF93EF93FF93EE
:1052B0008091A2059091A305892B29F0E091A20588
:1052C000F091A3050995FF91EF91BF91AF919F9147
:1052D0008F917F916F915F914F913F912F910F909F
:1052E0000FBE0F901F9018951F920F920FB60F923E
:1052F00011242F933F934F935F936F937F938F93DB
:105300009F93AF93BF93EF93FF938091A4059091E8
:10531000A505892B29F0E091A405F091A505099533
:10532000FF91EF91BF91AF919F918F917F916F917D
:105330005F914F913F912F910F900FBE0F901F9053
:1053400018951F920F920FB60F9211242F933F932F
:105350008F939F93AF93BF938091AA059091AB05D4
:10536000A091AC05B091AD053091AE050196A11D9F
:10537000B11D232F2D5F2D3720F02D570196A11D34
:10538000B11D2093AE058093AA059093AB05A09321
:10539000AC05B093AD058091A6059091A705A091AD
:1053A000A805B091A9050196A11DB11D8093A60580
:1053B0009093A705A093A805B093A905BF91AF91BD
:1053C0009F918F913F912F910F900FBE0F901F9043
:1053D00018958FB7F8942091AA053091AB054091AC
:1053E000AC055091AD058FBFB901CA0108959FB7B3
:1053F000F8942091A6053091A7054091A8055091F9
:10540000A90586B5A89B06C08F3F21F02F5F3F4FAF
:105410004F4F5F4F9FBF542F432F322F2227280F0C
:10542000311D411D511D82E0220F331F441F551FA6
:105430008A95D1F7B901CA010895EF92FF920F93AF
:105440001F93CF93DF937B018C010E94F729EB011F
:105450000EC00E94F7296C1B7D0B685E7340C8F379
:105460000894E108F10801091109C851DC4FE11461
:10547000F1040105110569F7CDB7DEB7E6E00C943C
:105480002930789484B5826084BD84B5816084BD00
:1054900085B5826085BD85B5816085BDEEE6F0E0AD
:1054A000808181608083E1E8F0E010828081826009
:1054B0008083808181608083E0E8F0E0808181608A
:1054C0008083E1EBF0E0808184608083E0EBF0E0BA
:1054D000808181608083EAE7F0E08081846080835E
:1054E0008081826080838081816080838081806808
:1054F00080831092C1000895CF93DF93482F50E02E
:10550000CA018D5F934FFC0134914151544FFA0110
:105510008491882369F190E0880F991FFC01EF5274
:10552000F44FA591B491FC01E552F44FC591D4918B
:10553000662351F42FB7F8948C91932F909589237B
:105540008C93888189230BC0623061F42FB7F89463
:105550008C91932F909589238C938881832B8883BA
:105560002FBF06C09FB7F8948C91832B8C939FBF5D
:10557000DF91CF910895833071F0843028F4813029
:10558000A1F0823021F514C08630B1F08730D1F01F
:105590008430E9F404C0809180008F7703C080914B
:1055A00080008F7D80938000089584B58F7702C03E
:1055B00084B58F7D84BD08958091B0008F778093EE
:1055C000B00008958091B0008F7D8093B000089561
:1055D000FF920F931F93F62E482F50E0CA01895E69
:1055E000934FFC012491CA018D5F934FFC011491EC
:1055F0004151544FFA0104910023C9F0222319F0BC
:10560000822F0E94BB2AE02FF0E0EE0FFF1FE55231
:10561000F44FA591B4919FB7F894FF2021F48C9199
:105620001095812302C08C91812B8C939FBF1F9179
:105630000F91FF9008950F931F93482F50E0CA01D8
:10564000895E934FFC012491CA018D5F934FFC0149
:1056500004914151544FFA011491112319F420E09F
:1056600030E015C0222319F0822F0E94BB2A812F1F
:1056700090E0880F991F8B51944FFC01A591B49134
:105680008C9120E030E0802311F021E030E0C9016E
:105690001F910F910895982F8E3008F09E509770AB
:1056A000809148038295880F880F807C892B809396
:1056B0007C0080917A00806480937A0080917A00E7
:1056C00086FDFCCF2091780040917900942F80E0F6
:1056D00030E0282B392BC9010895A0E0B0E0E3E7C2
:1056E000FBE20C940B307C016B018A01C0E0D0E03E
:1056F0000FC0D6016D916D01D701ED91FC91019024
:10570000F081E02DC7010995C80FD91F0150104045
:105710000115110571F7CE01CDB7DEB7E8E00C94A5
:105720002730EF92FF920F931F93CF93DF937C016B
:105730008B01C0E0D0E0F8010F5F1F4F649166233A
:1057400059F0D701ED91FC910190F081E02DC70156
:105750000995C80FD91FEFCFCE01CDB7DEB7E6E070
:105760000C942930DC01ED91FC910190F081E02D49
:1057700009950895EF92FF920F931F938C016DE0AE
:105780000E94B22B7C01C8016AE00E94B22B9C01EE
:105790002E0D3F1DC9011F910F91FF90EF900895AD
:1057A000EF92FF920F931F937C010E94912B8C012B
:1057B000C7010E94BA2B9C01200F311FC9011F9104
:1057C0000F91FF90EF900895EF92FF920F931F9328
:1057D0007C010E94B22B8C01C7010E94BA2B9C0154
:1057E000200F311FC9011F910F91FF90EF90089575
:1057F000CF93DF93EC016115710519F420E030E0DF
:105800000FC0DB010D900020E9F71197A61BB70B25
:10581000E881F9810280F381E02DAD0109959C01B9
:10582000C901DF91CF9108954F925F927F928F923D
:105830009F92AF92BF92CF92DF92EF92FF920F931F
:105840001F93DF93CF93CDB7DEB7A1970FB6F89430
:10585000DEBF0FBECDBF2C01742ECB01223008F469
:105860002AE019A231E2C32ED12CCC0EDD1E822EED
:105870009924AA24BB24672D752FA50194010E94A9
:10588000C42F79018A01C801B701A50194010E94C2
:10589000922F472D461B0894C108D1084A3010F4B6
:1058A000405D01C0495CF6014083E114F10401054B
:1058B000110521F07E2C5F2DC801DDCFC201B6019C
:1058C0000E94F82BA1960FB6F894DEBF0FBECDBF95
:1058D000CF91DF911F910F91FF90EF90DF90CF90CC
:1058E000BF90AF909F908F907F905F904F90089562
:1058F000DC012115310541F4ED91FC910190F0811D
:10590000E02D642F099508950E94142C0895EF92BC
:10591000FF920F931F937C010E94782C8C01C7018A
:105920000E94BA2B9C01200F311FC9011F910F91BA
:10593000FF90EF900895EF92FF920F931F939A01BB
:105940007B0100E010E0B801A7010E94782C1F91B4
:105950000F91FF90EF900895EF92FF920F931F9396
:105960007C010E949B2C8C01C7010E94BA2B9C01D8
:10597000200F311FC9011F910F91FF90EF900895E3
:10598000EF92FF920F931F939A01E62EFF2400E0FF
:1059900010E0B801A7010E94782C1F910F91FF9091
:1059A000EF900895EF92FF920F931F937C010E9456
:1059B000C02C8C01C7010E94BA2B9C01200F311F03
:1059C000C9011F910F91FF90EF900895A0E0B0E002
:1059D000ECEEFCE20C940B30EC016A017B0121152A
:1059E000310541F4E881F9810190F081E02D642FC7
:1059F00009951BC02A303105B1F477FF13C06DE261
:105A00000E94B22B8C0144275527BA014C195D091D
:105A10006E097F09CE012AE00E94142C9C01200F00
:105A2000311F04C02AE00E94142C9C01C901CDB78B
:105A3000DEB7E8E00C942730EF92FF920F931F93AC
:105A40007B019A010027F7FC0095102FB801A701F0
:105A50000E94E62C1F910F91FF90EF900895EF9216
:105A6000FF920F931F937C010E941C2D8C01C70194
:105A70000E94BA2B9C01200F311FC9011F910F9169
:105A8000FF90EF9008950E94F82B0895EF92FF92F7
:105A90000F931F937C010E94432D8C01C7010E942C
:105AA000BA2B9C01200F311FC9011F910F91FF904C
:105AB000EF90089508951F920F920FB60F92112440
:105AC0002F933F934F938F939F93EF93FF938091E7
:105AD000C00082FD1DC04091C6002091EF053091AD
:105AE000F0052F5F3F4F2F7330708091F10590913B
:105AF000F2052817390771F0E091EF05F091F005F4
:105B0000E155FA4F40833093F0052093EF0502C032
:105B10008091C600FF91EF919F918F914F913F919E
:105B20002F910F900FBE0F901F9018951F920F92FC
:105B30000FB60F9211242F933F938F939F93EF9360
:105B4000FF93209133063091340680913506909171
:105B500036062817390731F48091C1008F7D809374
:105B6000C10014C0E0913506F0913606ED50FA4FB1
:105B70002081809135069091360601968F73907042
:105B800090933606809335062093C600FF91EF91DF
:105B90009F918F913F912F910F900FBE0F901F906B
:105BA0001895A0E0B0E0E7EDFDE20C940730FC01B1
:105BB0001382128288EE93E0A0E0B0E084839583A4
:105BC000A683B7838BE893E091838083758764878E
:105BD00057874687318B208B138B028BF58AE48A9B
:105BE000D78AC68AB18EA08E938E828E8F85848F3F
:105BF0008889858F8989868F8A89878F8B8980A3F9
:105C00002096ECE00C942330AF92BF92DF92EF929B
:105C1000FF920F931F93CF93DF93EC017A018B01D7
:105C2000DD24403081EE580780E0680780E0780787
:105C300011F0DD24D39491E0A92EB12CEC89FD89DB
:105C4000DD2069F0C50108A002C0880F991F0A94E1
:105C5000E2F7808360E079E08DE390E005C0108298
:105C600060E874E88EE190E0A80197010E94C42FDB
:105C700021503040404050405695479537952795E4
:105C800080E12030380720F0DD2011F0DD24D6CF70
:105C9000E889F9893083EA89FB89208319A2EE8992
:105CA000FF89408121E030E0C9010C8C02C0880FDF
:105CB000991F0A94E2F7482B4083EE89FF894081BF
:105CC000C9010D8C02C0880F991F0A94E2F7482B76
:105CD0004083EE89FF894081C9010E8C02C0880F84
:105CE000991F0A94E2F7482B4083EE89FF8980814F
:105CF0000F8C02C0220F331F0A94E2F7209528234D
:105D00002083DF91CF911F910F91FF90EF90DF9053
:105D1000BF90AF900895DC011C96ED91FC911D970A
:105D2000E05CFF4F2191319180819181281B390BDB
:105D30002F733070C901089587E396E00E948B2E7F
:105D4000892B11F00E945A2D0895DC011C96ED91CB
:105D5000FC911D97E05CFF4F20813181E054F040C1
:105D6000DF01AE5BBF4F8D919C91119728173907CA
:105D700019F42FEF3FEF07C08D919C91E80FF91FA9
:105D80008081282F30E0C9010895DC011C96ED9137
:105D9000FC911D97E05CFF4F20813181E054F04081
:105DA000DF01AE5BBF4F8D919C911197281739078A
:105DB00019F42FEF3FEF10C08D919C911197E80FD0
:105DC000F91F20818D919C91119701968F7390708E
:105DD00011969C938E9330E0C9010895DC01919651
:105DE0008C919197882339F05496ED91FC915597B9
:105DF000808186FFF9CF91961C920895CF93DF930F
:105E0000EC01EE85FF85E05CFF4F20813181E0549D
:105E1000F0402F5F3F4F2F733070DF01AE5BBF4FFD
:105E20008D919C91119728173907D1F3E05CFF4FB2
:105E300080819181E054F040E80FF91F6083EE8586
:105E4000FF85E05CFF4F31832083EE89FF8920814D
:105E500081E090E00F8C02C0880F991F0A94E2F74E
:105E6000282B208381E089A3EC89FD8980818064CF
:105E7000808381E090E0DF91CF9108958F929F928F
:105E8000AF92BF92CF92DF92EF92FF920F931F9348
:105E900000D000D00F92EDB7FEB7319684E0ADB7D9
:105EA000BEB711968C9383E0818387E0828385E07F
:105EB000838381E0848387E396E06FEA75E043EFB4
:105EC00055E025EC30E004EC10E0B0ECEB2EF12CCA
:105ED000A1ECCA2ED12CF2ECAF2EB12CE6EC8E2E1A
:105EE000912C0E94D12D0F900F900F900F900F903A
:105EF0001F910F91FF90EF90DF90CF90BF90AF90E8
:105F00009F908F900895CF93DF930E94412A0E9423
:105F10000D28CCE9DEE20E9417122097E1F30E94DF
:105F20009C2EF9CF629FD001739FF001829FE00DFC
:105F3000F11D649FE00DF11D929FF00D839FF00D08
:105F4000749FF00D659FF00D9927729FB00DE11DB4
:105F5000F91F639FB00DE11DF91FBD01CF01112491
:105F6000089597FB092E07260AD077FD04D086D026
:105F700006D000201AF4709561957F4F0895F6F7CA
:105F8000909581959F4F0895A1E21A2EAA1BBB1BE5
:105F9000FD010DC0AA1FBB1FEE1FFF1FA217B307F5
:105FA000E407F50720F0A21BB30BE40BF50B661F0B
:105FB000771F881F991F1A9469F7609570958095CF
:105FC00090959B01AC01BD01CF01089597FB092E6F
:105FD00005260ED057FD04D0D7DF0AD0001C38F4B8
:105FE00050954095309521953F4F4F4F5F4F089505
:105FF000F6F790958095709561957F4F8F4F9F4FE5
:1060000008952F923F924F925F926F927F928F925C
:106010009F92AF92BF92CF92DF92EF92FF920F9337
:106020001F93CF93DF93CDB7DEB7CA1BDB0B0FB641
:10603000F894DEBF0FBECDBF09942A8839884888FE
:106040005F846E847D848C849B84AA84B984C88494
:10605000DF80EE80FD800C811B81AA81B981CE0F8B
:10606000D11D0FB6F894DEBF0FBECDBFED01089570
:10607000EE0FFF1F0590F491E02D0994AA1BBB1BA6
:1060800051E107C0AA1FBB1FA617B70710F0A61B38
:10609000B70B881F991F5A95A9F780959095BC0159
:1060A000CD010895911106C0803219F089508550B4
:0E60B000D0F70895992788270895F894FFCF18
:1060BE004E6F005965730054582074696D656F7585
:1060CE007421006D6F64756C65206C6F636B656415
:1060DE003F00486F70206368616E6E656C20002013
:1060EE0040200053004E2F4100386368002C002CD6
:1060FE00205B005D20280029004E4F5420454E4164
:10610E00424C45440053656E64696E672073657436
:10611E0074696E677320746F2052580A005265734B
:10612E00657474696E672073657474696E67732025
:10613E006F6E2052580A0041626F7274656420655A
:10614E00646974730A00696E76616C6964207365A4
:10615E006C656374696F6E000D0A496E76616C69C9
:10616E006420696E707574202D206469736361728A
:10617E006465642107007363616E6E6572206D6FD6
:10618E0064650053657474696E6773207361766518
:10619E006420746F20454550524F4D0A005265766B
:1061AE0065727465642073657474696E67732066B6
:1061BE00726F6D20454550524F4D0A004C6F616411
:1061CE00656420666163746F7279206465666175BB
:1061DE006C74730A004B657920616E64206368618C
:1061EE006E6E656C732072616E646F6D697A656434
:1061FE000A004F70656E4C52536E672054582073D0
:10620E0074617274696E672000206F6E204857208B
:10621E000050504D005253534900534441005343D4
:10622E004C00525844005458440041494E004C42D0
:10623E004545500053504B54524D00534255530058
:10624E0053554D44004C4C494E440000342B340001
:10625E003800382B340031320031322B34003136D5
:10626E000001000000C01200001A400AA1204EA535
:10627E00001B1E27522C23308025000005400AA14A
:10628E00204EA50020244EA52C2330004B000006E6
:10629E00400AD0009D49007B289D492C233000E107
:1062AE00000005400A4501D7DC03B81E0EBF0023CF
:1062BE002E48E801008A400A6001555502AD1E20A5
:1062CE00000023C88025000005400AA1204EA5002D
:1062DE0020244EA52C2330000200020002000200F2
:1062EE000200020002000200020002000200020090
:1062FE0002000200020002FF01610265026A026EE4
:10630E0002720276027A027E0284028B029002955B
:10631E00029B029B029B029B0235019C02A002A2E1
:10632E0002A602A902AE02350100070B0C101115D0
:10633E0000160A1322312900000000FE2E6D2B8B51
:08634E002EC52EA52EEE2E0037
:107E00000F92CDB7DEB7112484B714BE81FFF1D035
:107E100082E08093C00088E18093C10086E0809377
:107E2000C20080E18093C4008EE0CDD088249924E4
:107E3000CC24C394F5E0DF2EE1E1EE2E73E0F72EC3
:107E4000B6D0082F813479F4B2D08983C2D0898129
:107E5000823811F481E005C0813811F485E001C059
:107E600083E09ED09AC0823411F484E103C085344B
:107E700019F485E0B6D091C0853561F498D0082F0B
:107E800010E095D090E0982E8824802A912A880CC2
:107E9000991C82C0863521F484E0A3D080E0E1CF34
:107EA000843609F04CC083D082D0A82E80D0B82E62
:107EB00000E011E07CD0F80181938F01AE16D1F77C
:107EC00088D0FB2DF53489F4E0E0F1E00BC0F9999E
:107ED000FECF92BC81BC0894811C911C819180BD15
:107EE000FA9AF99AEA1598F358C08B2D863409F05E
:107EF00054C0F401F7BEE89507B600FCFDCFF401CD
:107F0000A0E0B1E02C9130E011968C91119790E0B7
:107F1000982F8827822B932B12960C01C7BEE895C9
:107F20001124329681E0A038B80761F7F401D7BE7A
:107F3000E89507B600FCFDCFE7BEE8952EC0843774
:107F4000F1F435D034D0182F32D0B82E42D0FB2DDA
:107F5000F63421F4F40105914F010CC0FB2DF534EA
:107F600049F4F999FECF92BC81BC0894811C911C04
:107F7000F89A00B5802F14D0115049F70EC08537FC
:107F800039F427D08EE10CD085E90AD08FE069CF93
:107F9000813511F488E017D01CD080E101D050CF9A
:107FA0009091C00095FFFCCF8093C600089580910A
:107FB000C00087FFFCCF8091C00084FD01C0A89560
:107FC0008091C6000895E0E6F0E098E19083808318
:107FD0000895EDDF803219F088E0F5DFFFCF84E10E
:107FE000DFCF1F93182FE3DF1150E9F7F2DF1F9166
:0E7FF0000895282E80E0E7DFEE27FF27099492
:027FFE0001057B
:0400000300007E007B
:00000001FF
